:020000020000FC
:060000000BC089C191C193
:10001400D7C1E8C100E806BD00E006BD0FED0DBF85
:1000240032E000E00ABB08E007BB00E601BB929A9D
:1000340095989698C39802E000BF00E003BF09E0DA
:1000440006BF0CBF01E00FBD08E00EBD00E808B913
:1000540000EF00BD00E20BBF789408E7CCD106B3F3
:1000640006950695069506950A95F4E0E4E1000FD9
:1000740010E0E00FF11F05911491F8010995FFCFED
:100084000BB700640BBF00E305BF829B03C0C3989A
:100094008895FBCFC39AF9CF0BB700640BBF00E37D
:1000A40005BF829B05C03F7D30FB31F98895F9CFB0
:1000B40035FDF7CF306231FF316031FD3E7F30FDD9
:1000C400C39A30FFC39830FDE4D030FFFDD0E9CFB0
:1000D4000CE205BF34600BB700680BBF8895FECFF8
:1000E4000CE205BF38600BB700680BBF8895FECFE4
:1000F40000E814E006BD16BD0BB700640BBF829B7D
:100104000AC03F7D30FB31F930FD0CE230FF0CE3D7
:1001140005BF8895F4CF35FDF2CF306231FF3160F1
:1001240031FD3E7F30FF16C010E002E01BBD0ABD6A
:1001340010E00DEF1DBD0CBD01E80FBD0DE00EBDBF
:1001440010E00CEF1DBD0CBD3061A3D00BB70068EF
:100154000BBFD5CF0BB70F770BBF0AB700680ABF29
:1001640001E00FBDC398B0D0CACF00E806BD01E0DE
:1001740006BD0BB700640BBF829B0AC030FB31F98C
:100184003F7D30FD00E230FF00E305BF8895F4CFEA
:1001940035FDF2CF306231FF316031FD3E7F30FFFB
:1001A4000FC0969A00E408B974D00FEF24D10FEF72
:1001B40022D108B1006108B908B1086008B9DCCFE0
:1001C40000E008B9969880D0D7CF58E061E078E78E
:1001D40084E128D056E062E07FEA84E623D057E049
:1001E40062E077ED87E81ED058E062E07BEE8EEDAA
:1001F40019D056E063E075EF8CEE14D057E063E05D
:100204007AEF82EF0FD058E063E07DEF85EF0AD0FC
:1002140055E065E07EEF88EF05D058E064E07EEFBE
:1002240088EF00D000E806BD56BD0BB700640BBFD5
:10023400829B0AC030FB31F93F7D30FD00E230FF84
:1002440000E305BF8895F4CF35FDF2CF306231FF6E
:10025400316031FD3E7F30FF17C010E01BBD7ABD19
:100264000EB5087F01600EBD10E00DEF1DBD0CBD85
:1002740010D00DBD8CBD0EB56770087F062B0EBD6A
:100284000FB5006C0FBDD4CF0FB50F730FBD1CD0CD
:10029400CFCF2FB7F89416B51F7000E806BD01E064
:1002A40006BD03B7016003BF00B7006100BF00E5EE
:1002B400A2D000B70F7E00BF03B70E7F03BF00E8D4
:1002C40006BD16BD2FBF08952FB7F89416B51F703D
:1002D40000E806BD01E006BD03B7016003BF00B737
:1002E400006100BF00E587D000B70F7E00BF04EBBC
:1002F40082D000B7006100BF00E57DD000B70F7E5B
:1003040000BF03B70E7F03BF00E806BD16BD2FBFB5
:1003140008950F931F930FB70F930F910FBF1F9162
:100324000F91189532FDC39A0F931F930FB70F9334
:1003340032FD05C033FD19C034FD28C039C00DECB1
:100344005AD00DEC58D00DEC56D00DEC54D00DEC29
:1003540052D00DEC50D00DEC4ED00DEC4CD00DEC39
:100364004AD00DEC48D0C39823C01FE00FEF2AB742
:1003740027FD05C00A95D9F71A95C1F719C0C39A84
:100384000DEC39D00DEC37D0C39812C00CB5033046
:1003940078F00B3E68F401E00FBDC39A04E62BD05D
:1003A400C39810E00CED1DBD0CBD01E80FBD00C0ED
:1003B4000AB700680ABF0F910FBF1F910F911895DC
:1003C4000F931F930FB70F93C39A0AEF14D00AEF3A
:1003D40012D0C39808B1006108B90F910FBF1F91E3
:1003E4000F91189517CE1895000014E01A95F1F79F
:1003F4000A95D1F708951F932F9312E022E02A95CE
:10040400F1F71A95D9F70A95C1F72F911F9108951D
:10041400F600E700FB00EC000001F10005010A0111
:0E04240072000F016A00B7004E007A0042001D
:00000001FF
